BL51 BANKED LINKER/LOCATER V5.03                                                        06/14/2006  18:23:33  PAGE 1


BL51 BANKED LINKER/LOCATER V5.03, INVOKED BY:
C:\KEIL\C51\BIN\BL51.EXE STARTUP.obj, main.obj, delay.obj TO ringtone1 RAMSIZE (256) CODE (0X0000-0X1FFF)


MEMORY MODEL: SMALL


INPUT MODULES INCLUDED:
  STARTUP.obj (?C_STARTUP)
  main.obj (MAIN)
  delay.obj (DELAY)
  C:\KEIL\C51\LIB\C51S.LIB (?C_INIT)
  C:\KEIL\C51\LIB\C51S.LIB (?C?ULDIV)
  C:\KEIL\C51\LIB\C51S.LIB (?C?ULSHR)


LINK MAP OF MODULE:  ringtone1 (?C_STARTUP)


            TYPE    BASE      LENGTH    RELOCATION   SEGMENT NAME
            -----------------------------------------------------

            * * * * * * *   D A T A   M E M O R Y   * * * * * * *
            REG     0000H     0008H     ABSOLUTE     "REG BANK 0"
            DATA    0008H     0004H     UNIT         _DATA_GROUP_
            DATA    000CH     0003H     UNIT         ?DT?MAIN
                    000FH     0011H                  *** GAP ***
            BIT     0020H.0   0000H.1   UNIT         ?BI?MAIN
                    0020H.1   0000H.7                *** GAP ***
            IDATA   0021H     0001H     UNIT         ?STACK

            * * * * * * *   C O D E   M E M O R Y   * * * * * * *
            CODE    0000H     0003H     ABSOLUTE     
                    0003H     0008H                  *** GAP ***
            CODE    000BH     0003H     ABSOLUTE     
                    000EH     07F2H                  *** GAP ***
            CODE    0800H     00E1H     UNIT         ?C?LIB_CODE
            CODE    08E1H     00A9H     UNIT         ?PR?TMR0?MAIN
            CODE    098AH     008CH     UNIT         ?C_C51STARTUP
            CODE    0A16H     0076H     UNIT         ?CO?MAIN
            CODE    0A8CH     005BH     UNIT         ?PR?_TONEGEN?MAIN
            CODE    0AE7H     002EH     UNIT         ?PR?MAIN?MAIN
            CODE    0B15H     0020H     UNIT         ?PR?_DELAYMS?DELAY
            CODE    0B35H     0013H     UNIT         ?PR?TMR0INIT?MAIN
            CODE    0B48H     0012H     UNIT         ?PR?_DELAYUS?DELAY
            CODE    0B5AH     000BH     UNIT         ?PR?NOTEPLAYSTART?MAIN
            CODE    0B65H     000AH     UNIT         ?C_INITSEG
            CODE    0B6FH     0007H     UNIT         ?PR?NOTEPLAYSTOP?MAIN



OVERLAY MAP OF MODULE:   ringtone1 (?C_STARTUP)


SEGMENT                          DATA_GROUP 
  +--> CALLED SEGMENT          START    LENGTH
----------------------------------------------
?C_C51STARTUP                  -----    -----
BL51 BANKED LINKER/LOCATER V5.03                                                      06/14/2006  18:23:33  PAGE 2


  +--> ?PR?MAIN?MAIN
  +--> ?C_INITSEG

?PR?MAIN?MAIN                  -----    -----
  +--> ?PR?TMR0INIT?MAIN
  +--> ?PR?_DELAYMS?DELAY
  +--> ?PR?NOTEPLAYSTART?MAIN
  +--> ?PR?NOTEPLAYSTOP?MAIN

*** NEW ROOT ***************************************************

?PR?TMR0?MAIN                  -----    -----
  +--> ?CO?MAIN
  +--> ?PR?_TONEGEN?MAIN

?PR?_TONEGEN?MAIN              0008H    0004H



SYMBOL TABLE OF MODULE:  ringtone1 (?C_STARTUP)

  VALUE           TYPE          NAME
  ----------------------------------

  -------         MODULE        ?C_STARTUP
  C:098AH         SEGMENT       ?C_C51STARTUP
  I:0021H         SEGMENT       ?STACK
  C:0000H         PUBLIC        ?C_STARTUP
  D:00E0H         SYMBOL        ACC
  D:00F0H         SYMBOL        B
  D:0083H         SYMBOL        DPH
  D:0082H         SYMBOL        DPL
  N:0000H         SYMBOL        IBPSTACK
  N:0100H         SYMBOL        IBPSTACKTOP
  N:0080H         SYMBOL        IDATALEN
  C:098DH         SYMBOL        IDATALOOP
  N:0000H         SYMBOL        PBPSTACK
  N:0000H         SYMBOL        PBPSTACKTOP
  N:0000H         SYMBOL        PDATALEN
  N:0000H         SYMBOL        PDATASTART
  N:0000H         SYMBOL        PPAGE
  N:0000H         SYMBOL        PPAGEENABLE
  D:00A0H         SYMBOL        PPAGE_SFR
  D:0081H         SYMBOL        SP
  C:098AH         SYMBOL        STARTUP1
  N:0000H         SYMBOL        XBPSTACK
  N:0000H         SYMBOL        XBPSTACKTOP
  N:0000H         SYMBOL        XDATALEN
  N:0000H         SYMBOL        XDATASTART
  C:0000H         LINE#         92
  C:098AH         LINE#         99
  C:098CH         LINE#         100
  C:098DH         LINE#         101
  C:098EH         LINE#         102
  C:0990H         LINE#         151
  C:0993H         LINE#         155
  -------         ENDMOD        ?C_STARTUP
BL51 BANKED LINKER/LOCATER V5.03                                                      06/14/2006  18:23:33  PAGE 3



  -------         MODULE        MAIN
  C:0000H         SYMBOL        _ICE_DUMMY_
  D:0090H         PUBLIC        P1
  D:00A0H         PUBLIC        P2
  C:0A16H         PUBLIC        noteDuration
  B:0020H.0       PUBLIC        notePlayEn
  B:00A8H.7       PUBLIC        EA
  B:0090H.6       PUBLIC        KEYUP
  C:0A8CH         PUBLIC        _ToneGen
  D:00CBH         PUBLIC        RCAP2H
  D:00CAH         PUBLIC        RCAP2L
  C:0AE7H         PUBLIC        main
  D:0089H         PUBLIC        TMOD
  C:0A50H         PUBLIC        noteFreq
  B:00A8H.1       PUBLIC        ET0
  B:0088H.5       PUBLIC        TF0
  D:008CH         PUBLIC        TH0
  D:00CDH         PUBLIC        TH2
  D:008AH         PUBLIC        TL0
  D:00CCH         PUBLIC        TL2
  B:00A0H.0       PUBLIC        LED
  B:0088H.4       PUBLIC        TR0
  B:00C8H.2       PUBLIC        TR2
  D:000CH         PUBLIC        noteIdx
  C:0B5AH         PUBLIC        notePlayStart
  C:08E1H         PUBLIC        Tmr0
  B:0090H.0       PUBLIC        BUZZER
  D:00C9H         PUBLIC        T2MOD
  D:00C8H         PUBLIC        T2CON
  C:0B6FH         PUBLIC        notePlayStop
  C:0B35H         PUBLIC        Tmr0Init
  D:000DH         PUBLIC        notePlayCtr
  B:0090H.4       PUBLIC        KEYDN
  -------         PROC          TMR0
  C:08E1H         LINE#         81
  C:08FEH         LINE#         83
  C:0901H         LINE#         84
  C:090CH         LINE#         85
  C:0914H         LINE#         86
  C:091AH         LINE#         87
  C:091CH         LINE#         88
  C:0932H         LINE#         89
  C:0932H         LINE#         90
  C:0949H         LINE#         91
  C:095FH         LINE#         92
  C:0961H         LINE#         93
  C:0963H         LINE#         94
  C:0965H         LINE#         95
  C:0967H         LINE#         96
  C:0969H         LINE#         97
  C:0969H         LINE#         98
  C:0969H         LINE#         99
  C:0969H         LINE#         100
  C:0969H         LINE#         101
  C:096CH         LINE#         102
  C:096FH         LINE#         104
BL51 BANKED LINKER/LOCATER V5.03                                                      06/14/2006  18:23:33  PAGE 4


  -------         ENDPROC       TMR0
  -------         PROC          TMR0INIT
  C:0B35H         LINE#         116
  C:0B35H         LINE#         117
  C:0B35H         LINE#         119
  C:0B38H         LINE#         120
  C:0B3BH         LINE#         122
  C:0B3EH         LINE#         123
  C:0B41H         LINE#         125
  C:0B43H         LINE#         126
  C:0B45H         LINE#         127
  C:0B47H         LINE#         128
  -------         ENDPROC       TMR0INIT
  -------         PROC          _TONEGEN
  D:0006H         SYMBOL        tone
  -------         DO            
  D:0008H         SYMBOL        tmp
  -------         ENDDO         
  C:0A8CH         LINE#         146
  C:0A8CH         LINE#         147
  C:0A8CH         LINE#         149
  C:0A90H         LINE#         150
  C:0A90H         LINE#         151
  C:0A93H         LINE#         153
  C:0A96H         LINE#         154
  C:0A99H         LINE#         156
  C:0AB0H         LINE#         157
  C:0AC6H         LINE#         158
  C:0AD4H         LINE#         159
  C:0AD9H         LINE#         160
  C:0ADCH         LINE#         161
  C:0ADFH         LINE#         163
  C:0AE1H         LINE#         164
  C:0AE2H         LINE#         166
  C:0AE2H         LINE#         167
  C:0AE4H         LINE#         168
  C:0AE6H         LINE#         169
  C:0AE6H         LINE#         170
  -------         ENDPROC       _TONEGEN
  -------         PROC          NOTEPLAYSTART
  C:0B5AH         LINE#         186
  C:0B5AH         LINE#         187
  C:0B5AH         LINE#         188
  C:0B5DH         LINE#         189
  C:0B5FH         LINE#         190
  C:0B64H         LINE#         191
  -------         ENDPROC       NOTEPLAYSTART
  -------         PROC          NOTEPLAYSTOP
  C:0B6FH         LINE#         206
  C:0B6FH         LINE#         207
  C:0B6FH         LINE#         208
  C:0B71H         LINE#         209
  C:0B73H         LINE#         210
  C:0B75H         LINE#         211
  -------         ENDPROC       NOTEPLAYSTOP
  -------         PROC          MAIN
  C:0AE7H         LINE#         218
BL51 BANKED LINKER/LOCATER V5.03                                                      06/14/2006  18:23:33  PAGE 5


  C:0AE7H         LINE#         219
  C:0AE7H         LINE#         220
  C:0AEAH         LINE#         221
  C:0AECH         LINE#         223
  C:0AECH         LINE#         224
  C:0AECH         LINE#         225
  C:0AEFH         LINE#         226
  C:0AEFH         LINE#         227
  C:0AF6H         LINE#         228
  C:0AF9H         LINE#         229
  C:0AFCH         LINE#         230
  C:0AFFH         LINE#         231
  C:0B01H         LINE#         232
  C:0B01H         LINE#         233
  C:0B01H         LINE#         235
  C:0B04H         LINE#         236
  C:0B04H         LINE#         237
  C:0B0BH         LINE#         238
  C:0B11H         LINE#         239
  C:0B13H         LINE#         240
  C:0B13H         LINE#         242
  -------         ENDPROC       MAIN
  -------         ENDMOD        MAIN

  -------         MODULE        DELAY
  C:0000H         SYMBOL        _ICE_DUMMY_
  D:0090H         PUBLIC        P1
  D:00B0H         PUBLIC        P3
  D:00A8H         PUBLIC        IE
  C:0B15H         PUBLIC        _DelayMs
  D:00B8H         PUBLIC        IP
  C:0B48H         PUBLIC        _DelayUs
  D:0098H         PUBLIC        SCON
  D:0088H         PUBLIC        TCON
  D:00C8H         PUBLIC        T2CON
  D:00D0H         PUBLIC        PSW
  -------         PROC          _DELAYUS
  D:0006H         SYMBOL        N
  -------         DO            
  D:0004H         SYMBOL        x
  -------         ENDDO         
  C:0B48H         LINE#         36
  C:0B48H         LINE#         37
  C:0B48H         LINE#         40
  C:0B59H         LINE#         41
  -------         ENDPROC       _DELAYUS
  -------         PROC          _DELAYMS
  D:0006H         SYMBOL        msec
  -------         DO            
  D:0004H         SYMBOL        x
  D:0002H         SYMBOL        y
  -------         ENDDO         
  C:0B15H         LINE#         54
  C:0B15H         LINE#         55
  C:0B15H         LINE#         58
  C:0B1FH         LINE#         59
  C:0B1FH         LINE#         60
BL51 BANKED LINKER/LOCATER V5.03                                                      06/14/2006  18:23:33  PAGE 6


  C:0B2DH         LINE#         61
  C:0B34H         LINE#         62
  -------         ENDPROC       _DELAYMS
  -------         ENDMOD        DELAY

  -------         MODULE        ?C?ULDIV
  C:083CH         PUBLIC        ?C?ULDIV
  -------         ENDMOD        ?C?ULDIV

  -------         MODULE        ?C?ULSHR
  C:08CEH         PUBLIC        ?C?ULSHR
  -------         ENDMOD        ?C?ULSHR

*** WARNING L16: UNCALLED SEGMENT, IGNORED FOR OVERLAY PROCESS
    SEGMENT: ?PR?_DELAYUS?DELAY

******************************************************************************
* RESTRICTED VERSION WITH 0800H BYTE CODE SIZE LIMIT; USED: 022AH BYTE (27%) *
******************************************************************************

Program Size: data=16.1 xdata=0 code=892
LINK/LOCATE RUN COMPLETE.  1 WARNING(S),  0 ERROR(S)
